:080000001AC0FECFFDCFFCCFBA
:10000800FBCFFACFF9CFF8CFF7CFF6CFF5CFF4CFB4
:10001800F3CFF2CFF1CFF0CFEFCFEECFEDCFECCFE4
:10002800EBCFEACFE9CFE8CFE7CFE6CF0000F894EF
:10003800EE27EFBBE5BFF8E1A895A4B7A77FA4BF5B
:10004800F0936000E09360008DE0A2E0BB27ED93A1
:100058008A95E9F780E092E0A0E0B1E0ED9301979E
:10006800E9F7E4E3F0E085919591009761F0A591B7
:10007800B59105901590BF01F00105900D9201977B
:10008800E1F7FB01F0CFE0E0EEBBE0E0EABDE0E045
:10009800EBBDEFEFEDBFE2E0EEBFC0E8D1E016C088
:1000A800E881E066E0937C00E0917A00E064E09308
:1000B8007A00E0917A00E071E1F3E0917A00E06182
:1000C800E0937A00E091790021960895E0E8E093C2
:1000D8006100E0E0E0936100EFEFE5B9E4B9ECEF2F
:1000E800E8B9E0E0E7B9EBB9EFEFEAB9E0E0E4BD81
:1000F800E5BDE6BDE7BDE8BDE0938000E093810083
:10010800E0938500E0938400E0938700E093860005
:10011800E0938900E0938800E0938B00E0938A00E5
:10012800E093B600E093B000E093B100E093B20032
:10013800E093B300E093B400E0936900EDBBE09373
:100148006800E0936E00E0936F00E0937000E0E8D1
:10015800E0BFE0E0E0937B00E8E3E0937E00E0E6C8
:10016800E0937C00E3E8E0937A00E2E0EA9398DF2A
:100178004E2EEAE04E1608F42AC0E0E0EA9390DF3B
:100188003E2EE1E0EA938CDF2E2E732C8824E22D9C
:10019800F0E07E0E8F1EA72DB82DEAE0F0E02DD0FE
:1001A8007E2E8F2E231418F4E32DE21902C0E22DBF
:1001B800E3196E2E662011F4552406C0E62DA72DEE
:1001C800B82DF0E022D05E2EE4E6E51510F4E4E662
:1001D8005E2E5BB8E8ECF0E0FA93EA9302D0C5CF64
:1001E800FFCFE991F991309639F080ED97E00197CA
:1001F800F1F7A8953197C9F70895FA9FF02DEB9F6D
:10020800F00DEA9FE02DF10D08950024112490E1EE
:10021800AA0FBB1F001C111C0E1A1F0A18F40E0E81
:100228001F1E01C0A1609A9599F7FD01D00108959C
:00000001FF
